:1000000033C04DC04CC04BC04AC049C048C047C0B7
:1000100046C045C044C043C042C041C040C03FC0CC
:100020003EC03DC03CC03BC03AC039C038C037C0FC
:1000300036C035C057524F4E470A004F4B210A0079
:100040005472792025690A0052656164792E0A008C
:1000500045464765666700202B2D2E3031323334FC
:10006000353637383968000011241FBECFEFD4E091
:10007000DEBFCDBF11E0A0E0B1E0E2EFF5E002C0ED
:1000800005900D92AE30B107D9F711E0AEE0B1E0C6
:1000900001C01D92A431B107E1F709D0A8C2B0CFC9
:1000A0008091C00087FFFCCF8091C6000895AF9279
:1000B000BF92CF92DF92EF92FF920F931F93CF9355
:1000C000DF9383E390E080D000D088E490E0EDB748
:1000D000FEB7928381830AD2C0E0D0E00F900F90E8
:1000E00020E4A22E20E0B22E08EC10E09BE3C92E03
:1000F00090E0D92E84E3E82E80E0F82E00D000D0E6
:10010000EDB7FEB7B282A182D483C383EFD10F9043
:100110000F900F900F908091C00087FFFCCF8091CF
:10012000C600813329F58091C00087FFFCCF809104
:10013000C6008433E9F48091C00087FFFCCF809132
:10014000C6008733A9F48091C00087FFFCCF80915F
:10015000C600813369F480E29EE4F8013197F1F73B
:100160000197D9F700D0EDB7FEB7D282C1820CC09B
:1001700080E29EE4F8013197F1F70197D9F700D0BA
:10018000EDB7FEB7F282E182B1D10F900F9006C0B9
:100190008091C00087FFFCCF8091C6008091C00095
:1001A00087FDF6CF2196AACF1F93182F8A3011F41E
:1001B0008DE0FADF8091C00085FFFCCF1093C60070
:1001C00080E090E01F91089528E12093C100809382
:1001D000C400892F990F990B8093C50080E091E0AE
:1001E00090931101809310010895ABE0B0E0EAEF25
:1001F000F0E012C15C014B017A01FC01178216820A
:10020000838181FD08C06FEF7FEFFEC042E050E0C8
:10021000E40EF51E04C03E010894611C711CF5013A
:10022000D380F401D3FC8591D3FE81914F018823C3
:1002300009F4E7C0853259F4D3FC6591D3FE61918E
:100240004F01653219F0062F10E01AC085E290E0E8
:1002500029C0002309F4D5C087E590E0602F70E045
:100260000ED1892B39F4033211F4106103C00C361E
:1002700061F41068F401D3FC0591D3FE01914F01A4
:1002800017FFE7CF002309F4BCC080E590E0602FA2
:1002900070E0F5D0892B49F044E050E0E40EF51E03
:1002A0008FE390E0B501F6D0BACF033629F00337DB
:1002B00071F00335E1F40AC087010E5F1F4FF701AB
:1002C00080819181B501E6D07801A9CF1160F70155
:1002D000C080D18003C090E0B501DCD0F60110FDF4
:1002E000859110FF81916F018823A9F78FCF043684
:1002F00011F0093639F517FF08C0F7012081318167
:100300004281538184E090E00AC0F70180819181AD
:100310009C01442737FD4095542F82E090E0E80E81
:10032000F91E1F7E57FF08C05095409530952195C6
:100330003F4F4F4F5F4F1064CA01B901A3012AE03C
:1003400030E034C00037A9F0013730F40835B1F09F
:100350000F3609F056C006C0053739F0083709F0E6
:1003600050C008C028E030E00CC01F7E2AE030E01A
:1003700008C01061146220E130E003C0146020E185
:1003800032E017FF08C0F70160817181828193819B
:1003900044E050E008C0F70180819181BC0180E019
:1003A00090E042E050E0E40EF51EA301C2D0D82E4A
:1003B000D618012F10E006FF04C08DE290E0B501D1
:1003C00069D004FF13C0FE01ED0DF11D8081803363
:1003D00069F080E390E0B5015DD002FF07C00072D4
:1003E0001070C801885A9F4FB50154D0DA94F301B8
:1003F000ED0DF11D808190E0B5014CD0DD20B1F70D
:100400000ECFF50166817781CB012B96EEE020C0FF
:100410002F923F924F925F926F927F928F929F9214
:10042000AF92BF92CF92DF92EF92FF920F931F9302
:10043000CF93DF93CDB7DEB7CA1BDB0B0FB6F894B3
:10044000DEBF0FBECDBF09942A88398848885F84F3
:100450006E847D848C849B84AA84B984C884DF8064
:10046000EE80FD800C811B81AA81B981CE0FD11D48
:100470000FB6F894DEBF0FBECDBFED010895FC01AD
:100480000590061621F00020D9F7C0010895319794
:10049000CF0108950F931F93CF93DF938C01EB014E
:1004A0008B8181FF1BC082FF0DC02E813F818C811B
:1004B0009D812817390764F4E881F9810193F98354
:1004C000E88306C0E885F985802F0995892B31F4EA
:1004D0008E819F8101969F838E8302C00FEF1FEF55
:1004E000C801DF91CF911F910F910895A0E0B0E076
:1004F000EBE7F2E09DCFFE01359661917191A091FD
:100500001001B091110113968C9113978860139686
:100510008C938091100190911101AF0166DEE09102
:100520001001F09111012381277F23832096E2E0BF
:100530009BCFFA01AA27283051F1203181F1E894AC
:100540006F936E7F6E5F7F4F8F4F9F4FAF4FB1E0C6
:100550003ED0B4E03CD0670F781F891F9A1FA11DC1
:10056000680F791F8A1F911DA11D6A0F711D811DC2
:10057000911DA11D20D009F468943F912AE0269F87
:1005800011243019305D3193DEF6CF010895462FE6
:100590004770405D4193B3E00FD0C9F7F6CF462FC7
:1005A0004F70405D4A3318F0495D31FD4052419330
:1005B00002D0A9F7EACFB4E0A695979587957795ED
:1005C0006795BA95C9F700976105710508959B0174
:1005D000AC010A2E06945795479537952795BA95FD
:1005E000C9F7620F731F841F951FA01D0895F8940B
:0205F000FFCF3B
:0E05F2000000000200000000D4000000000025
:00000001FF
